S123800088090B05000000007E893C7EA1517EB9200032021E400022A00030000101017EAC
S12380200100000200006001000000320000000000000000000000000000000000000000A6
S1238040000000000000000000000000000000000000000000000000000000000000B2BEAC
S12380600000000000FFFFFF0000000000003200000000000032000000000000323FFFFF2C
S12380800000000000000000000000150100000000000000000000F00000000000000000D6
S12380A00000000000B76FB4FE00000000110BF00F0F00DA60000000000000008225822532
S12380C0A24A00000000A1BC00000000000000FFFFFFFFFFFFFFFFFFFFFFFFFFFFFFFFFF64
S12380E0FFFFFFFF00C00000FFFFFF01B80AAB2AFFFFFFFF0102040810204080FEFDFBF743
S1238100EFDFBF7F000000000000000000000000000000000000000000000000000000004F
S123812000000000000000000000000000000000000000000000000000000000000000003B
S1238140FFFFFFFFFFFFFFFFFFFFFFFFFFFFFFFFFFFFFFFFFFFFFFFFFFFFFFFFFFFFFFFF3B
S1238160FFFFFFFFFFFFFFFFFFFFFFFFFFFFFFFFFFFFFFFFFFFFFFFFFFFFFFFFFFFFFFFF1B
S12381800000000000000000000000000000000000000000000000000000000000000000DB
S12381A00000000000000000000000000000000000000000000000000000000000000000BB
S12381C0FFFFFFFFFFFFFFFFFFFFFFFFFFFFFFFFFFFFFFFFFFFFFFFFFFFFFFFFFFFFFFFFBB
S12381E0FFFFFFFFFFFFFFFFFFFFFFFFFFFFFFFFFFFFFFFFFFFFFFFFFFFFFFFFFFFFFF009A
S123820000000000000000010010200002000104080C05090D060A0E070B0F8081828300AE
S123822000000803000000000000000000000000000000000000000000000000000000002F
S1238240FFFFFFFFFFFFFFFFFFFFFFFFFFFFFFFFFFFFFFFFFFFFFFFFFFFFFFFFFFFFFFFF3A
S1238260FFFFFFFFFFFFFFFFFFFFFFFFFFFFFFFFFFFFFFFFFFFFFFFF8280827C1011010AE6
S123828000000000000000000000000034010F4E1A50964E2607109E5926040F383581ECB3
S12382A0A4DD592602DD5B1CAFADB80220E2E624C024CE804F1F98444444C4078E80FCE683
S12382C085E4C6E7C6A625974DE624A627BD87389E452721D17D251DA705E706967D8024B1
S12382E034028D6886FFB781062452CB24E706F781067E84239E472721D17D241DA705E748
S1238300066FE28D4786FFB781052431CB24D17D242BE706F781057E84239E3D272D10A31A
S1238320052624D64DE709CE803DBD86F6CE8043BD87228641A707EE04A64326098640A730
S1238340071F12BD8E0539AE8420D139CE804F4F5FA6C0260ECB08C14026F6EEE432631CA4
S1238360FE6EC434024F67E4240CE1632508EE6132641A016EC45C4C810826EA326120D75B
S1238380E624C024CE804F1F98444444C4078E80F4E685EAC6E7C6E624D17D2520A69F80D4
S12383A0A52718F181062504BD873839F781068601B781049E4527377E841B201EA69F80DD
S12383C0A72718F181052504BD873839F781058602B781049E4727177E841B7F8104A6270C
S12383E09E41270B10A30526022018AE8420F39E39270CBD8432CE8039BD86F67E84439EEB
S123840041270A8D2DCE8041BD86F620369E3D27FE8D1FCE803DBD86F6202827128D13A6D7
S1238420072A0AEE0C1F12BD8BCD7E8C3420317E83EFEC24A706E708A627A7056F8818BD4D
S1238440873839B6810481002608CE803FBD8722200E810126049F452006810226029F47CE
S12384608680A7071F12BD8E45BD8D03EE2CBD8BCDEE2CAE2E1A108603AAA841A78821A7D4
S123848088228603AAA84CA78823A788246FA8173410BD8C34EE2CAE2EBD8A781A106CA880
S12384A01931A8378D1F326231A8C9AE2AA60B270333C818EC2EC30002340631A8428D0521
S12384C032621CAF39AEC4EC81DD49EC81DD4BAF22AE62DC496F88C16F88C2A701E7884197
S12384E0DC4BA702E78842EC44ED24EC46ED26EC42ED28A6482747A6C8142705CC88A6200A
S123850003CC8894EDA4EC2210A3422513EC44ED22EC42A3C4C1022607DC49A702E788425D
S1238520A6C814270BEC4410A3C4260486012002860FAA2AA7882284FEA788212040EC42EF
S1238540A3C4C102260ECC88E3EDA4860AAA2AA78821202AC1042615CC88DEEDA4860BAAF5
S12385602AA78822860EAA2AA788212011CC88C2EDA4860FAA2AA7882284FEA7882139A681
S123858027E6249E3D271010A3052607A625A788182022AE8420EE9E45270C10A305260720
S12385A0A625A78818200E9E47260A10A3052605A625A78818BD873839AE24A68817260774
S12385C06C8817BD8738392002AE24A626BD8738A18819270139BD8BC1CE00009C45260614
S12385E0DF458D3320239C472606DF478D512019A6072A08CE803DBD86F6200D8540270840
S1238600CE8041BD86F62001398600A707CE803BBD8722BD88443986613402CE8056C61FA9
S1238620A6E4917D25111F98A4C4A7C4542504C67F335F6AE420E9350286FFB7810639867A
S1238640243402C6FECE804FA6E4917D24111F98A4C4A7C45825043341C6FE6CE420E935BD
S12386600286FFB7810539CE804F6FC01183805623F886FFB78106B7810539A625BD873828
S1238680109E41271AE627C501270FA125260B3402BD8E058640A727350210AEA420E439B6
S12386A0AE243430109E3D2726ECE410A324261ABD8E051F218640A707CE803DBD86F6CECB
S12386C08043BD8722109E3D200310AEA420D8BD8667109E45270AECE410A3242603BD8E1C
S12386E005109E47270AECE410A3242603BD8E053530BD873839344033423440EE0227108D
S123870010AE8410AFC42604EFF42002EF22200F10AE8410AFF8022704EF222002EFF432B3
S1238720643910AEC42604AF5E2002AFA4AFC410AF02CE0000EF84391A503402B6820726B7
S123874019DE57109F57EFA4965D4C975D81042309966427050F64BD89761CAF3582BDAE08
S1238760178E80386F808C805725F986FFB78105B78106CC8107DD571F01C30008ED841F25
S1238780018C81FF26F4861F975DB78207CC0000ED848EB0529F391F101F13C3004DED844E
S12387A09F3B3406BD884435061F01EF021083B2BA25E4CC0000FDB054CC0000EDC439CE73
S12387C082AE200F3402965D8104220235823502CE83801E107E87F7CE857F20F6CE867BC4
S12387E02015CE86A02010CE85C920081F31CE85B93088C9A6881934011A50BD881F9E5BB8
S1238800270510AF842003109F59109F5BCC0000EDA49638270235810A381CAF7E829010F9
S12388209E5726103456BD9F60BD9F6F1A500A38355620EBAF24ED26EF22AEA49F570A5D10
S12388407F82073910AE0E8603AA8841A7A821A7A8228603AA884CA7A823A7A824399E5E09
S123886010EF818CB2C625038EB2BE9F5E10EE84394F1F02EEA988BB57108EEC5F31A5AD85
S1238880D41CBF1A40F6ECE02B070C6026E3BDF1BB0F603BAE42EC81A721E7A841AC462642
S12388A002AE44AF4239AE42EC81A721E7A841AC46260C8601AA4AA7A821CC88A5A7C4AF7F
S12388C04239AE42EC81A721E7A841AF42AC48260CCC88DEEDC4860BAA4AA7A82139CC88A8
S12388E0E320F18E88A5AFC48603AA4AA7A8214F58C4F81F02EEA988BC7E87ECB089B089A3
S1238900B094B094B0D6B0D6B0E1B0E1B123B123B12EB12EB170B170B17BB17BB1BDB1BDC1
S1238920B1C8B1C8B20AB20AB215B215B257B257B262B262B2A4B2A4B2AFB2AF1A40B6E2A1
S12389400D2A1F850427037E8989852027037EF4DF8502270DB6E201962527050CE9BDA1CC
S1238960163BF6ECE02B037E88713B8D09CC89A1DD61B6E20A3934011A50B6E20C84FDB7E0
S1238980E20C8A0EB7E20C3581F6E20A1CBFAD9F80611A50965D810425048DDA20020A6406
S12389A03BC1902607CC8A25DD61203FC1802607CC89ECDD612034C1B826199628260E8671
S12389C001976BC67FBDA0DABDADB62005861BBDA4042017C1B926139628260F0F6B5FBD56
S12389E0A0DABDADB68E8068BD87DD39CB24D763CC89F6DD61398EFBFEE6859614801E34B0
S1238A0002EBE02802C67F2E02C6019663CE89A1DF61BDA0C5BDADBC96638E80680D1C27E7
S1238A20037E87BF39CB24D763CC8A2FDD61398EFBF8E6859614801E3402EBE02802C67F69
S1238A402E02C6019663CE89A1DF61BDA0B9BDADBA96638E80680D1C27037E87C4398EB0AE
S1238A6052108EEC7FCEE4188D2330884D31248CB2BA25F44FA75F3934601E121F2083ECB2
S1238A807F5454CEE41833C58D033560391A50EC881A6E981CE3881E2505A18820250ACC7A
S1238AA08AAEED881CA688205FED881A2029A388212505A18823220ACC8AD7ED881CA6888A
S1238AC0235FED881A2010A388242408CC8AD7ED881C4F5FED881A1CAFA188272303A6886C
S1238AE027E68828BDF5E71A50EC88296E982BE3882D2505A1882F2511CC8B0FED882BA6E8
S1238B00882F44A7882DA6882F5FED88292072A388302505A188322215CC8B81ED882B5F20
S1238B20A68832272C44A7882DA688322016A1882D22116488306688316C8831340244A73E
S1238B40882D3502ED88292038A3883325034D2617CC8BBEED882B5F4FED88293470BD8736
S1238B60E7EC882935702019A1882D22116488336688346C8834340244A7882D3502ED881B
S1238B8029E688362611D61EC1092605E688182003E69804582002C00158250F34463D8BB0
S1238BA007A761A6E48B07A7E4200E3442533D8B073402A6618B07A761BDF6DD35401CAF8E
S1238BC0398640A78824CC8AC7ED881C39E626D17D2502C0184F4CC00C2AFB4ACB0C8E8B39
S1238BE0F1E6858303B1E3492A014FEDA8107E8CA000152B40556B8095ABC0D5EB8E8068F3
S1238C00FC8011E301ED0530078C807D25F2108EB0520C4EBD8C3431A84D3420BD828C104A
S1238C20AEE4108CB1862603BD885E3520108CB2BA25DF39EE24E6A8142614961D81092614
S1238C4005E6A8182002E6448EF77DE68520015AA6A813ABA812A7A8128EF8CDA6862A055C
S1238C60403D4020013D1F891DE345E3A810BDF5143406EBA81589003406AE2EBDF5F1392A
S1238C80108EB052CC8AD7EDA81C6FA81ACC8BBEEDA82B6FA82931A84D108CB2BA25E5399B
S1238CA0AE2AA62680182A014FE6083D46563404E6A8161DEBE08900EB068900EB4C8900AC
S1238CC027072A035F2002C6FFD765A6A81AA0A8269B65240286FFA7A81AA6A820A0A826ED
S1238CE09B65240286FFA7A820A6A823A0A8269B65240286FFA7A823E7A826A64D8B39A747
S1238D00A82739AE2AEE2CB680158CB76F240C4881802204867F2001402005482A02867FB5
S1238D208B20E64B58583D9767A6289765A62680249766E603C10127058110240157E7A8BE
S1238D4015A607A7A828A601A7A813A602A7A8146FA812A605270E8004D66548583D4CAB26
S1238D6004240286FFA7A8364F5FEDA829EDA81AA7A826CC8A95EDA81CCC8AEFEDA82BCEBC
S1238D80F7FDBD8DA1300A312FBD8DA131319667E6A82F3DA7A82F9667E6A8323DA7A83219
S1238DA039A68811D6653D40AB0C8D4AEDA81EA68812D6653DAB0D2A014F811F2302861FEA
S1238DC03402484848A7A820A68813D6663D4067E467E4A0E08B08AB0E8D1BEDA821A6882A
S1238DE014D6653DAB0F2A014F811F2302861F484848A7A823392A034F2006811F230286D5
S1238E001F48ECC639AE2ACEF7FDCC8AC7EDA81CCC8B49EDA82BE629A688153D40AB881022
S1238E208DD4EDA824E629A6881F3D40AB881AE6A82954E7A82D545454C0083404A0E08D1E
S1238E40B5EDA83339E626C1242402C624C1612302C661CE8E4DA6C5840FD17D24079EA784
S1238E60CE8EAF20059EA5CE8EBFAF2AEEC6EF2C390000000000000000000000000000007F
S1238E800000000000000000000000000000000000000000000000000000000000000000CE
S1238EA0000000000000000000000000000000B31EB336B34EB366B37EB396B3AEB3C6B5D1
S1238EC08FB5A7B5BFB5D7B5EFB607B61FB637109EA78E8EAFCE8E714F8D113402109EA51D
S1238EE08E8EBF8D0735028B24977D39E62A58AE85A10E2205E7C64C20F7308818CB026D41
S1238F002B2705308818CB02813C2204C10E23E13934264F108CB58F25028640977EBD988A
S1238F20EB35268E8FF9EEA4C1082602A7A5C10F2609A1A8102221A7A5200AC110261DA13C
S1238F402F2315A7A56F2886FFA7A813A6A8104AA7A811A7A812202FBD994139C111260B51
S1238F60A12F25F4A1A81222EFA7A5C1122611A1A81125E4A1A81022DFA7A586FFA7A81352
S1238F80C1132603A7A813A62F0F816D28271BA1A811270A977FA6A8129780BD8FC80C8179
S1238FA0EF24A6A811E6A8122003E6A810977FD780BD8FC8EF26EF229681E6A8135C2701F7
S1238FC04FA7A814BD994139967FA7C08A805F4425045C4420FA967FAB850D8127079180ED
S1238FE023035A20F1CB08E685DA7EE7C0918024074C977F0F8120D239000103070F1F3FCE
S12390007F0009121B242D363F400000000000962F2A070C2FBD8A5E2003BD885E20F0BD28
S1239020885E96302AF90F30BD9039BD885E96302AF90F30BD8BFD20E61A50B6E20084FB01
S12390408A08B7E2001CAFB6ECE1B6ECE2BD885E1A50F6ECE2B6E2008A0CB7E2001CAFF7B5
S1239060900C4FFB900D8900FB900E890047564756B6ECE1B6ECE2F0900A2A07CB082B01C3
S12390805F2005C0082A015FCB402802C67F2A015FF19009270DF79009BDA0CFBDADAF8DD2
S12390A01FDD69FC900CFD900DF6ECE254F1900B270DF7900BD768D76CBDA0E2BDADB23995
S12390C086ABC0402A053D802B2006C13F26015C3D58D613492A053D901320013D47564783
S12390E05639BD9D4B8D0220F996AE810A2404BD92583996AE8110250881172204BD943B6D
S12391003996AE81182504BD95F0398D09810E27D8810F27D43996AE810B2608BDAB90BDF6
S123912092492007810C2613BD9249D68BBD9D2DCEFB4DA6C6E6C5DDB34F39810D2609BD24
S123914092490C83BD998B39810E260C0D8327F29788860197842012810F1026003A0D839A
S123916027E0978886809784200086C8978796879732BD998B7D820827024F39BD9D4B965E
S12391808891AE26120D3226F3C614D18727DFD687C03CD78720D739810A102600A99682D3
S12391A0810410260096968581032601398104260E96E781062606BDAB60BD96F44F39815A
S12391C0082610BD9FB40DBA2B06BD92497E912B0FBA398101261A0D8C27169690C6033DAD
S12391E03404D68C5AEBE08E82099691EA86BDA0F2BD9E837D80072707BD9249BD9431394A
S1239200D685C101262E96912704810127169690978FC6243D108EB4FE31AB109FA79691AC
S1239220810226109690978EC6243D108EB76F31AB109FA5BD8ECF8D1016FEEF96828105B3
S123924026058D0516FEE44F390F820F850F830F840F330F8A0F8939108EFB4D9682810058
S1239260102600440DAE271C0DA42604C61C2002C67C96AE978DA6A6DDB3BD94310F8A866C
S1239280019782390DA42609D68F5CE6A5861C2007D68E5CE6A5867CDDB3CC80059783D763
S12392A082860197890F8A39810110260088BD9249D6AEE6A5D7B4968DC60A3DDBAEC10BB8
S12392C0250ECE9FF3A6C5270781FF2707D78B39BD943139D78B1F98810B26085FD792C6F9
S12392E01C7E92FB810C2609C601D792C67C7E92FB810D2614C602D792C6EE86B6DDB3860B
S12393000297859782BD943139810E2610CCB6CEDDB3BD9431CC09049785D78239810F26F3
S123932004BD9F9A3981102604BD9F9A39CC2A3ADDB3BD9431398102261096AE2607969140
S123934081022713398103230E398103262E96AE2704810925013996858101270481052681
S123936004C6102002C605A6A5D6AED78CE6A5DDB30F900F8A0F898604978239810426205E
S123938096AE8101251981042215D685C101260F0D8C270BE6A64A9790968CA6A6DDB339B8
S12393A081051026006C0DAE260E0DA427050FA416FED10CA416FECC96AE810125548104C9
S12393C02250E6A6D7B44ABD9249C680D7830D1626040DA42710978EC6243DC3B76FDDA592
S12393E00D16270C968E978FC6243DC3B4FEDDA7BD8ECF1A50BD875E1CAFD6AE5A0D162790
S123940004CB0C200A0DA42604CB1C2002CB2CBDA0F28106261A96AE81012514810422109C
S1239420E6A6D7B44A97B7CC08049785D7820F8939CC0180978A9789D78339CEFB4D96AEE0
S12394408110270481112653860197859682262086029782861CD6AEC1102709C61CDDB306
S12394600F917E95DDC67CDDB3860197917E95DD9691810226013996828102261E96AE8139
S1239480112707969181012606399691260139CC1CEEDDB3860297917E95DD96AE811227F0
S12394A00681131026008696AE81122608C67C860197A42004C61C0FA486B6DDB3860397A4
S12394C085CC03E8DD34BD9431BD9DD7DC34270220F7BD9F60BD9700BD974EC61FF7E201C7
S12394E01E891E89F6E201C4C0C140260686029793200EC1802705B7E20120DCBD9795972D
S123950093BD9F6FBD9249CEFB4D9693270D81012613CC2AB6DDB3BD943139CCB68EDDB38C
S12395208680978339860B97AEBD91163996AE8114102500AB8117102200A596AE81152633
S12395403B8604978596E781002606BD95E139202281022609BDAB90BD95E139201581047E
S12395602611BDAB80CC3A7ADDB3868097830F8A0F8939BDAB90BD95E139205D8114262F63
S12395808604978596E78104260EBDAB53860497820F8A0F8939200981002605BDAB4E2078
S12395A006BDAB90BDAB4EC604D782860A202A8116260C8603978286059785861C201A8187
S12395C01726160DE427088602978286072006C603D7828606978586B6C6B6DDB3BD94312C
S12395E039BDAB438657978B860D97AEBD91163996AE81192609BD9249BD96F41600F48198
S12396001A1026000A860C97AEBD91161600E4811B1026003796E781002604BD95E1398199
S123962006260ABDAB60BD9249BD96F43981082613BDAB9096272704BD95E139860C97AE2B
S1239640BD911639BDAB9020F31600A7811C1026001096E78100270481022603BD95E116A0
S12396600091811D1026000E96E781002606BDAB45BD95E4207D811E2609860B97AEBD91D7
S12396801620704D2B0139843F1F89444444448E820CA6869791C40F8E820FE6852B261FB6
S12396A098840397905454D78CCC01049785D782860A97AE8E8023A68434126F84BD90E970
S12396C03512A78439C4035CD7AE96163402969126060FA40F16200E8101260697A40F16EA
S12396E0200486019716860597820FB3BD96B43502971639CCB60ADDB38680978339FF18F8
S12397001A508614B7E200BDAE178EE41F9618BBB2838B5B240286FFB796FE108E03E8BDD5
S1239720F0A7D61926058610B7E200BD98585F96174A48FDE206CC4CC0B7E20BF7E20E8D25
S12397400139FC96FEE784E710A784A718398DF2CEECE2E6C486140F980F990F9A8D1C4A6C
S123976026FBC603D19A2312D199230CD19823048607200286032002860639E6C4CB802AF4
S12397800150C17F25020C9AD11A25020C99C10825020C9839961B263B96A4260C0FAABDEF
S12397A09A858E03FA861E200A0FA9BD9A858E038E863C6F4A6F4BC6083436AF29A72E6FF1
S12397C02F6F28CCFF10BD8F11353631A8185A26E8BD8ECFBD986C2B14969BB7E2005D2A58
S12397E009C47FB7E200969C20014F200C847F9794969CB7E200C47F4FF798479E94C62831
S1239800E72BCEECE20F99108E000131212603860139BD977B0D9927F2C606F7E20F108E34
S1239820E20413E6A44D271413E6A4E6C426015CE7808C800025F1A73C8E000013E6A4E6D2
S1239840C426015CE7808C00F025F1CC1000E7804A26FBBD99414F39B6E20084FCD6A4273E
S1239860028A02979B4C979CB7E20039BD9A85EC0FD7969794391F318C80002404969B2056
S12398800630898000969CB7E2003341E684391F21B6E2008C80002404969B2006969C30DE
S12398A0898000B7E2003121E784398D3EBD986CDE96335F1F328DBE3404335E8DB88DCF74
S12398C0313E109C9426F335048DC48D74398D1BBD986CDE941F328D9D34048D998DB011F6
S12398E0939626F735048DA78D5739BD9858BD986C6D28274BA6A811A12F27255F1F0333F0
S12399005FBD9876261B315F33579E9430083410BD9876BD988F335E313E10ACE424F1327A
S123992062BD9A85DE9610AEA812312130C8103410BD98766F84BD988F11A3E426F3326274
S123994039BD9A85A6282742BD9858BD986CEE26ECA812A15E2606C1802402C6FFA1A810DF
S12399602609C1DF2305C6DF6FA814E7A813EEA8123341109E9630A8103410BD98766F8430
S1239980BD988F10ACE426F3326239CE9FF3D68BA6C597AC1F89C43F848097AB0FA10FA397
S12399A0860197A2968B811E26068E801C7E9CC1968B811B102500BB813B102200B58D0213
S12399C0200C0DA42704109EA539109EA739968B811B10260018302A860797A00CA30D84F8
S12399E0102702DDBD9CC1BD8ECF3916005F811C10260012302B0D84102702C9BD9CC1BDC1
S1239A008ECF39160047811D102600140D841027005534261A50BD875E1CAF352616002D7B
S1239A20812210260006BD9D41160021812310260006BD9D41160015812410260006BD9D90
S1239A4038160009812510260003BD9D41968B812D250781312203BD9D41968B81372507BF
S1239A60813B2203BD9D418EA057A68597A030A57E9CC1968B813C102500B481481022000D
S1239A80AE8D02201C96A4270A108E8EBFDEA596A92008108E8EAFDEA796AA48AEA61F129C
S1239AA03930859F9D968B813C251C814022180D84270D2B05A6844C2003A6844ABD8F11FF
S1239AC09E9DE6847E9D15968B814126150D84270C2B04860120014FC608BD8F119E9D7EC1
S1239AE09CD3968B8142261A8E809F0D84270E2B076C84BD98AB20056A84BD98CEE6841684
S1239B000213968B8146270481472603BD9D38968B8148260E860197A30D8427068D04BDAB
S1239B208ECF39CEA077C008A6C597A07E9CC1968B815125608158225C815126058E802067
S1239B4020508152260B860197A3D7A08E80212041815326058E80222038815426078E802E
S1239B6023D7A0202D815526058E80242024815626058E8025201B81572610BD9D3886C627
S1239B8097A0860197A18E80262007815826038E80277E9CC1968B8118260D8E8015BD9DF4
S1239BA038867E97A07E9CC1811926068E80167E9CC1811A26140F9F0DA427058E80A92057
S1239BC0038E80AA860197A3201E8115260A866397A08E80121600E9811626058E801320BF
S1239BE007811726088E8014D7A07E9CC18149260E861E97A1866397A08E80171600C281A8
S1239C004A260DBD9D3886C697A08E80181600B1814B26068E80191600A7814C260DBD9D8B
S1239C20388E801A867E97A0160096814D26068E801B16008C814E26058E801D20AA814F55
S1239C4026068E801E16FFA08150260CBD9D388E801F867E97A020698159261A0D8427108B
S1239C602B0C860197280F6BBD87DD7E9C700F288E80287E9CD3815B26058E8029204281C3
S1239C805C26158E802A0D84270C2B07860BB7E20620037FE2062029816126070F848E8048
S1239CA02B201E816226070F848E80072013816326070F848E80062008BD9431CC111220DB
S1239CC0620DAB271A0D84270A2B068601A78420026F84CC12116D842602C60F7E9D230D43
S1239CE08427182B0CE684D1A02410DBA2E784200AE684D1A12304D0A2E784E68496A3279B
S1239D000E2B035C200981812603542002545496AC8440270C1F9844444444840FC40F20AF
S1239D20028D0ACEFB4DA6C6E6C5DDB3394FC10A2505C00A4C20F739868197A3860297A2E4
S1239D4039868297A3860497A23900B69D4A81002636BD9DD796AF810B2704811126099789
S1239D60AD8602B79D4A204996AF81F0271697AD860597318601B79D4A108EFB68D6ADA6CA
S1239D80A597AE3920CC204C81012621BD9DD7963126F996AF81F026F386059731BD9DD711
S1239DA0963126F98600B79D4A20A7202781022623BD9DD796AF91AD260C108EFB68A6A688
S1239DC097AE200F200D860D97AE860597318601B79D4A3916FF7BDCB30D832B0626034C00
S1239DE020015C97B5D7B65F86F097AFD7B21F988A180D8A270AC680D533260408B52006E9
S1239E0008B5240284F70D89270AC680D533260408B6200608B6240284EF1F89CA18F7E203
S1239E200F1E121E12F6E20FC4E0C1E02602C60FD7B1B7E20F86019737BD885EBDA41A24BF
S1239E401597AE8601B78208BD90E97F8208860F97B186F097AF0D372705BD885E20F79644
S1239E60B1810F2714860208B124034A20F997B0D6B258DBB2DBB0D7AFD6B25CC1071023F3
S1239E80FF6A3996858101261FB68223B7821F96912708810126088602205F8601205B96E2
S1239EA08C2704860320533F8102261AB68223B7821F96922708810126088605203C8604BE
S1239EC020388606203481052604860720068106260A8608F68222F7821F201E8107260977
S1239EE0C603F7821F860A201181092605860B5F2008860FB780077E9F1BD68CF1821F234D
S1239F0008860EB780077E9F1BFD8220BD9F60FC8220BDA4352504BD9F6F39BD9F6FB6806E
S1239F2007273B81012605CC7A9E202F8102250981052205CC2A8E202281062605CC387A80
S1239F40201981072605CC2A7A201081082605CCCE7A200781092606CC2A1ADDB33920FED5
S1239F601A50BDAB90BDF1BBBD8C80BDF541391A50BDF541BDF52DBD875EBD896BBDA07EB3
S1239F8086CCB7E20B7FE2067FE2077FE2047FE2050F790F6B0F721CAF3997BA810F26049B
S1239FA0861C2002867CC69CDDB3BD94310F8AC606D7823996B7C6243DDDB8BD99C21F210B
S1239FC0D6BA2722C10F2607DCB8C3B4FE2009C1102613DCB8C3B76F1F038600C6241F023B
S1239FE0BDF55B0FBA39CC2A3ADDB3868097BABD9431390000000000000000000000FFFF7E
S123A000FFFFFFFF00000000090C3F208107098B80810102030405060708000C0D0E0F1045
S123A0201112131415161718191A1B1C1D1E1F4F505152538840094A0B0C0D0E0909810936
S123A04081090909810F810381810981810081810000000040204001636363FC7CC6A00491
S123A0600700011F1F1F1F1F7C7C7C7C7C1F1F1F1F1F7C7C7C7C7C0107FF3FC6C63C86032F
S123A080B7E1008695B7E100CC8225DDBCDDBECCA1BCDDC6CCA24ADDC07F82357F82367FBD
S123A0A08237393446DCBC93BE2A0150C1082305BD885E20F035C68DEA34011A50DDC2C6B2
S123A0C090205F8DDE34011A50DDC2C680205334011A504FDDC2C6E0201234011A50864041
S123A0E0200634011A508601DDC2C6B09623274420301A509623810227048103260E3404C6
S123A100C6C0D7BBDA218D3035048D2C1CAFDCBC1093BE26F93934011A50C6F8D7BB8D18C9
S123A1203581DA21D1BB2704D7BB8D0CD6C28D08D6C38D04DCC2358196222701399EBCE783
S123A140808C823525038E82259FBC86B5B7E100393476B6E1002A518530271DB682372729
S123A1600297CEBDA094B6E1018E80766F03BD87DD8E8076BD87E22030850127288D5C1A02
S123A18040B68236B18235270F8E8238E6864C843FB782368D6F20E77F823796CE27040F64
S123A1A0CE20C020048502260D35763B3506DDC0393506DDC639AD9F80C620ED9EBEA680E0
S123A1C0B7E1018C823525038E82259CBC260996222600C695F7E1009FBE39F6E101B68204
S123A1E037271FB682358E8238E7864C843FB78235B18236260532627EA163326235763B1B
S123A20020037C823796222703BDA13D1CBF5D2B046E9F80C0D7C5C470C1702720D6C5C40A
S123A2200FD7C496202607D12127037EA247D6C5C4705757578EA3D4EC85DDC039D6C5C48B
S123A2400F8EA3E4586E95BDA1AC398D43BDA1ACCEA24BDFC0C1002602C64096C4BDADBC95
S123A26096C48E80767E87BF8D26BDA1ACCEA268DFC096C4C100260DC640BDADBC96C48EA2
S123A28080767E87BFBDADBA96C48E80767E87C4C1242404CB0C20F8C1602304C00C20F80D
S123A2A0D7C439C1402606CCA32BDDC039C160261196CD8180250BBDA4040FCDBDA1AC7E74
S123A2C0A341D11D2704D11E2608D7C4CCA30DDDC039CEA341DFC0962191C42610C17C267D
S123A2E0040F20200CC17D2604D7202004C17B26068E80767E87E239BDA1ACCEA2F8DFC05B
S123A30096232708BDADAFBD90C0DD77398D329623271796C427138108240F911E2602D7EA
S123A32076911D2605D77ABDADB2398D149623270FBDADB6C440D77926068E8076BD87DD4F
S123A34039CEA2A3DFC039BDA1AC96231027FEF758961F3D1F89961D81082602D77A961E8B
S123A36081082602D77620DFBDA1AC96231027FED6D7C4BDA1AC58961F3D1F89961D81093A
S123A3802706961E8109260896C48E8076BD87D820D6BDA1ACC12F22F9CA8096238102266F
S123A3A0071F98BDA404200681032602D7CD20E296252609962427050CE9BDA11639861CEA
S123A3C02006861E2002861DD6242707D6252603BDA40439A24BA268A36BA2A3A395A34A91
S123A3E0A2F8A24AA247A247A247A247A247A247A247A247A3B0A247A3BEA3C6A3C2A24737
S123A400A3D3A3D334011A10BE8278A7808C828C25038E827CBF82783581BE827ABC8278E1
S123A42026031CFE39A6808C828C25038E827CBF827A1A0139BDA4BAB68007810027031600
S123A4400064B680CF81012605BDA4D4205881022605BDA4D4204F81032605BDA4D4204699
S123A46081042605BDA53A203D81052605BDA53A203481062605BDA53A202B81072605BD85
S123A480A5A1202281082605BDA5FC201981092605BDA5A12010810A2605BDA5FC20078141
S123A4A00B2603BDA653B6E801B78002B68007810026041CFE20021A0139B780CFF780D011
S123A4C0BDAB207F800786E81F8BBDF08FB68002B7E80139BDF4C68640B4E2008100260803
S123A4E08607B7800716004EBDA8B9B68007810027031600417F80E17F80E3B680CF810183
S123A5002707B680CF81032614B6E20084FCB7E200BDA69CB68006810027022019B680CF72
S123A52081022707B680CF8103260BB6E20084FCB7E200BDA6E8BDF4D639BDF4C68640B4FF
S123A540E200810026088607B7800716004F8602B780E17F80E3B680CF81042707B680CFF7
S123A56081062614B6E20084FCB7E200BDA69CB68006810027022025B680CF81052707B6CC
S123A58080CF81062614B6E20084FCB7E200BDA6E8B68006810027022003BDA97CBDF4D639
S123A5A039BDF4C68640B4E200810026088607B78007160043BDA8B9B68007810027022093
S123A5C037B680CF81072606108EFBA8200881092604108EFBC87F80E3BDAAD2B680068131
S123A5E0002705BDAB0020107F80E1BDA847B6800681002703BDAB00BDF4D639BDF4C686FB
S123A60040B4E200810026088607B7800716003FB680CF81082606108EFBA82008810A26BD
S123A62004108EFBC87F80E3BDAAD2B6800681002706BDAB001600178602B780E1BDA847CB
S123A640B6800681002705BDAB002003BDA97CBDF4D639BDF4C68640B4E2008100260886D8
S123A66007B780071600318602B780E3108EFB88BDAAD2B6800681002705BDAB002019B60E
S123A68080D6B780038E8011BF8004BDF476B6800681002703BDAB00BDF4D639108EFB9065
S123A6A0BDAAD2B6800681002706BDAB001600377F80DD8602B780DE7F80E0B680E18100CE
S123A6C02605BDA736200781022603BDA78BB6800681002705BDAB00200DBDA7AEB6800623
S123A6E081002703BDAB0039108EFB9CBDAAD2B6800681002706BDAB001600398602B7803C
S123A700DDB780E08604B780DEB680E181002605BDA736200781022603BDA78BB6800681C6
S123A720002705BDAB00200DBDA7AEB6800681002703BDAB0039B680D6B78003B6E200BA22
S123A74080DDB7E2008E0000BF8004BDF448B6800681002703160032B680E08100260B8EB0
S123A760B31DCC0271C3B31D200D810226098EB58ECC0271C3B58EFD80DB108E0000A6A002
S123A780A780BC80DB26F77C80D639B680D6B78003B680E0810026058EB31D200781022619
S123A7A0038EB58EBF8004BDF4767C80D639B680D6B78003B680D5B78002B6E200BA80DD13
S123A7C0B7E2008E0000BF8004B680E181002605BDF448200781022603BDF476B680068198
S123A7E000270220617C8003B68003810527058C800026D2B680038105261A7F80037C80C0
S123A80002B68002B180D7220CBDF07DB68006810027022031B68002B180D722058C8000F0
S123A82026A4B68002B180D722078C80001026FF957C80DDB68002B180D7220AB680DDB102
S123A84080DE1026FF7439B680D6B78003B680D5B78002B680CF81072707B680CF810826BB
S123A86008CC0800C3B8002006CC2000C3B800FD80DB8EB800BF8004B680E181002605BD8F
S123A880F448200781022603BDF476B680068100270220247C8002B68002B180D7220CBD2B
S123A8A0F07DB6800681002702200DB68002B180D72205BC80DB26BD397F80E2BDAA2FB64D
S123A8C0800681002706BDAB001600AFB680CF810310260018F680D05A8EFBDFA685B480D5
S123A8E0D281002605C604F7800716008E81071026005CB680D08101253DB680D08103223A
S123A900368EFBEAF680D05AA685B480D4810026138EFBE2A685B480D381002605C605F7F2
S123A92080072011B680E427078609B780CF20058609B7800720158EFBE2F680D05AA68521
S123A940B480D381002605C605F7800716002C8EFBD4B680CFF680D05C5C3DA685B480D2E7
S123A96081002617B680CF81012607C603F78007200981022605C602F78007397F80E2BD26
S123A980AA2FB6800681002706BDAB0016007BB680CF810610260012F680D05A8EFBDFA675
S123A9A085BA80D2B780D216004E8108102600158EFBE2F680D05AA685BA80D3B780D3BDB7
S123A9C0AA0B160033810A102600158EFBEAF680D05AA685BA80D4B780D4BDAA0B160018A8
S123A9E08EFBD4B680CF1CFE8203F680D05C5C3DA685BA80D2B780D28602B780E2BDAA2FA0
S123AA00B6800681002703BDAB0039F680D05AB680CF8108260D8EFBF0A685B480D4B78066
S123AA20D4200B8EFBEDA685B480D3B780D339108EFB8C8602B780E3BDAAD2B6800681006B
S123AA40270316008CB680D5B78002B680D6B780038E80D2860AB78001B680E28100260A2B
S123AA60BDF013B6E803A784200781022603BDF0377A8001B680012707B68006810026D973
S123AA80B680068100271EBDF086BDF07DB680E28100260ABDF013B6E803A7842007810254
S123AAA02603BDF037B6800681002702202330017C8002B68002B180D7220CBDF4A4B68034
S123AAC00681002702200AB68002B180D71023FF8839B680E381002605B680D120058102F1
S123AAE026014F30A6A680B780D5B78002A680B780D6A680B780D7A684B780D8BDF4A4396D
S123AB008601B780078610B5800627078606B78007200C8640B5800627058608B780073945
S123AB20F780D05A5858F780D139B7A2FEB804A6C0DFEC97F139FEB808FFB804A7C0DFEE8D
S123AB400FF0398DE70F360FE9C602D7E739860497E739DEE5335DDFEC8DDBC606D7E739BF
S123AB600F360FE90CEB0FEA86609726860897E7F69009BDADAFD66CBDADB2D66B7EADB6CD
S123AB800F360FE9BDAC108DA38DABC60AD7E73996E7277B0FE7DEEE8106260686FF203261
S123ABA020498108263E96F00D2427260DEB26ECD6EAC10C240890EA24028B18201450CBE2
S123ABC0183404ABE0240B4CA75F8681A7C086FFA7C0A75F8680A7C0A7C0A7C0FFB806BD00
S123ABE0AB2C2007810A2603BDAC27CEAB2ADFEE8D4D8E806FBD87E2CE8E4D8624E6C62AF9
S123AC0009C47FE7C6C640BDA0C34C816125EE39BEB806DEE5FFB806BCB8042306A682A72B
S123AC20C220F5FFB804399EECDEEEDFEC96F09BF1A75FA680A7C09CE525F8FFB806395F8C
S123AC40D772BDA0DA5D26068E806FBD87DD39CCD800FDC00010B3C000260497E4DDE5962F
S123AC60E7273BD62426208104271A810627160D362712D6E8DB26D7E82406BDACA3BDA12F
S123AC80160A3620EC20170DE92713BDACA396EA4C811826034F0FEB97EA0AE920EBBD8840
S123ACA05E20BC96E78102260D0DF12607BDACEB0DF120F7202C810A261696F12610BDAC56
S123ACC0EBDCF281802703BDAD8F96F120EE20128108260D96F081FF26058681BDAD9A20B4
S123ACE001391A500AF10CF01CAF39DEECA64297F1ECC43343DFECDDF22A56847F81022F82
S123AD0017BDA0B7108E8E4DE6A6CA80E7A6D6F38E806FBD87C420374D2708D7F1335FDFCE
S123AD20EC202C9627271C0FF196E7810A260C335DDFECBDAB90BDAB842006BDABF2BDAB76
S123AD402C200C335DDFECBDAB90861ABDA404203D81032317BDA0C5108E8E4DE6A6C47FBA
S123AD60E7A6D6F38E806FBD87BF20228100260ABDA0CFBD90C0DD70201481012609D77351
S123AD80D76FBDA0E2200781032603BDAC40398181261AD6F0DBF1250139DEEE1193EC25C0
S123ADA00139A7C1DFEED6F0E75D0FF039200D4F200A86012006860320028A8034011A5037
S123ADC0DEEE1193EC250E35013404BDAB90861ABDA4043584EDC496E78108260C96F0A7A6
S123ADE05F3343DFEE0FF0202C810A260C96F0A75F3343DFEE0FF0201C81062618A6C481EB
S123AE008325126F5F3343DFEE3404BDAB608619BDA40435043581CEE418CC0000BDF5E741
S123AE201183E42026F7CEB052CC8AD78E8BBEEDC81CAFC82B6FC81A33C84D1183B2BA2554
S123AE40EE39ACFF16002B7C8003B68003810626E37C80027CA242B680028150240DBDAE10
S123AE60F0B6800681002703160007B6A242810126BF39B6800397028688B78000970013DF
S123AE809603A78020F9B6800397028688B78000970013960320FBB68003970286A8B78029
S123AEA000970013A680970320F9B68003970286A8B78000970013A684970320F986E8B728
S123AEC080009700139603A78020F986F8B78000970013A680970320F9860CB780009700D3
S123AEE020FEB680029703861CB78000970020FE8658B78000970020FE8678B7800097003A
S123AF0020FE86D0B780009700D600C50126FAF78006108E00011700013912121212313F0A
S123AF2026F839326CD600F78006B6800081882707B6800081E8260AF68006C45CF7800670
S123AF402020B6800081A82707B6800081F8260AF68006C45CF780062008F68006C418F7B1
S123AF60800639FFFFFFFFFFFFFFFFFFFFFFFFFFFFFFFFFFFFFFFFFFFFFFFFFFFFFFFFFF2B
S123AF800000000000000000000000000000000000000000000000000000000000000000AD
S123AFA000000000000000000000000000000000000000000000000000000000000000008D
S123AFC0FFFFFFFFFFFFFFFFFFFFFFFFFFFFFFFFFFFFFFFFFFFFFFFFFFFFFFFFFFFFFFFF8D
S123AFE0FFFFFFFFFFFFFFFFFFFFFFFFFFFFFFFFFFFFFFFFFFFFFFFFFFFFFFFFFFFFFFEF7D
S123B00000000000000000000000000000000000000000000000000000000000000000002C
S123B02000000000000000000000000000000000000000000000000000000000000000000C
S123B040FFFFFFFFFFFFFFFFFFFFFFFFFFFFFFFFFFFF00000000806800000000B4FEB31E93
S123B060EC7F0200001004010000000000000000000000000000000000000000000000004A
S123B0800000000000000000000000000000000000000000000000000000000000000000AC
S123B0A0000000806800000000B4FEB31EEC8302000010040100000000000000000000009B
S123B0C000000000000000000000000000000000000000000000000000000000000000006C
S123B0E010000000000000000000001000000000806800000000B4FEB31EEC87020000103C
S123B100040100000000000000000000000000000000000000000000000000000000000026
S123B1200000000000000000000000000020000000000000000000002000000000806800E3
S123B140000000B4FEB31EEC8B0200001004010000000000000000000000000000000000DA
S123B16000000000000000000000000000000000000000000000000000003000000000009B
S123B18000000000003000000000806800000000B4FEB31EEC8F020000100401000000007E
S123B1A000000000000000000000000000000000000000000000000000000000000000008B
S123B1C00000000000000040000000000000000000004000000000806800000000B4FEB39E
S123B1E01EEC93020000100401000000000000000000000000000000000000000000000097
S123B20000000000000000000000000000000000000000005000000000000000000000508A
S123B22000000000806800000000B4FEB31EEC970200001004010000000000000000000005
S123B2400000000000000000000000000000000000000000000000000000000000000000EA
S123B260006000000000000000000000E000000000806800000000B4FEB31EEC9B02000096
S123B280100401000000000000000000000000000000000000000000000000000000000095
S123B2A00000000000000000000000000000F000000000000000000000F0000000000000AA
S123B2C0FFFFFFFFFFFFFFFFFFFFFFFFFFFFFFFFFFFFFFFFFFFFFFFFFFFFFFFFFFFFFFFF8A
S123B2E0FFFFFFFFFFFFFFFFFFFFFFFFFFFFFFFFFFFFFFFFFFFFFFFFFFFFFFFFFFFFFF0069
S123B300000000000000000000000000000000000000000000000000000000000032B3DE66
S123B320B3E0B3DEB3E00002000000BE1E00000000F000000000B3FEB41EB3FEB41E00007E
S123B340000000BE1E00010001F000000000B41EB43EB41EB43E0000000000BE1E000100B6
S123B36001F000000000B43EB45EB43EB45E0000000000BE1E00010001F000000000B45EF0
S123B380B47EB45EB47E0000000000BE1E00010001F000000000B47EB49EB47EB49E00005D
S123B3A0000000BE1E00010001F000000000B49EB4BEB49EB4BE0000000000BE1E00010056
S123B3C001F000000000B4BEB4FEB4BEB4FE0000000000BE1E00010001F000000000000062
S123B3E00100FFFFFFFFFFFFFFFFFFFFFFFFFFFFFFFFFFFFFFFFFFFFFFFFFFFFFFFF4037ED
S123B400000000000000000000000000000000000000000000000000000000000000803771
S123B420000000000000000000000000000000000000000000000000000000000000C03711
S123B440FFFFFFFFFFFFFFFFFFFFFFFFFFFFFFFFFFFFFFFFFFFFFFFFFFFFFFFFFFFFFFFF08
S123B460FFFFFFFFFFFFFFFFFFFFFFFFFFFFFFFFFFFFFFFFFFFFFFFFFFFFFFFFFFFFFFFFE8
S123B4800000000000000000000000000000000000000000000000000000000000000000A8
S123B4A0000000000000000000000000000000000000000000000000000000000000000088
S123B4C0FFFFFFFFFFFFFFFFFFFFFFFFFFFFFFFFFFFFFFFFFFFFFFFFFFFFFFFFFFFFFFFF88
S123B4E0FFFFFFFFFFFFFFFFFFFFFFFFFFFFFFFFFFFFFFFFFFFFFFFFFFFFFFFFFFFF000E58
S123B5000001FC00000404000000010C0C040C0000000000021E14180A00000000000000A3
S123B5200000000C0001FC00000004000000011F0A0C0C0000000000011F14181900000053
S123B540000000000000000802013C000000030000000A1F1818180000000000021E1418E0
S123B56019000000000000000000000802013C000000030000000A1F1818180000000000F3
S123B580021E14181900000000000000000032B64FB651B64FB6510004000000BE1E000117
S123B5A00001F000000000B66FB68FB66FB68F0000000000BE1E00010001F000000000B63E
S123B5C08FB6AFB68FB6AF0000000000BE1E00010001F000000000B6AFB6CFB6AFB6CF0027
S123B5E000000000BE1E00010001F000000000B6CFB6EFB6CFB6EF0000000000BE1E000148
S123B6000001F000000000B6EFB70FB6EFB70F0000000000BE1E00010001F000000000B7DA
S123B6200FB72FB70FB72F0000000000BE1E00010001F000000000B72FB74FB72FB74F00BF
S123B64000000000BE1E00010001F00000000000000101FFFFFFFFFFFFFFFFFFFFFFFFFF23
S123B660FFFFFFFFFFFFFFFFFFFFFFFFFFFFFF403FFFFFFFFFFFFFFFFFFFFFFFFFFFFFFF65
S123B680000000000000000000000000000000803F000000000000000000000000000000E7
S123B6A0000000000000000000000000000000C03F00000000000000000000000000000087
S123B6C0FFFFFFFFFFFFFFFFFFFFFFFFFFFFFFFFFFFFFFFFFFFFFFFFFFFFFFFFFFFFFFFF86
S123B6E0FFFFFFFFFFFFFFFFFFFFFFFFFFFFFFFFFFFFFFFFFFFFFFFFFFFFFFFFFFFFFF0065
S123B700000000000000000000000000000000000000000000000000000000000000000025
S123B720000000000000000000000000000000000000000000000000000000000000000005
S123B740FFFFFFFFFFFFFFFFFFFFFFFFFFFFFFFFFFFFFFFFFFFFFFFFFFFFFFFFFFFFFFFF05
S123B760FFFFFFFFFFFFFFFFFFFFFFFFFFFFFF000C0001FC00000004000000181F18181848
S123B7800000000000051E1418180A0000000000000000000C0001FC000000030000000127
S123B7A01F0A0A0A0000000000011F0A140A000000000000000000000802013C00000003B6
S123B7C00000000A1F1818180000000000021E141819000000000000000000000802013C48
S123B7E0000000030000000A1F1818180000000000021E141819000000000000000000006C
S123B80001393939B80AB835B80A00C94000004000010000030018494000CB40184B40006B
S123B820C74018474000BB40183B4000C24060424000808080004D6972616765204F7065D3
S123B840726174696E672053797374656D20636F70797269676874203139383420456E7385
S123B8606F6E697120436F72702E202020627920416C6578204C696D62657269732C204A59
S123B8802E2057696C6C69616D204D617563686C792C204A6F686E204F2E2053656E696FFE
S123B8A07220616E6420416C616E20536D697468202020200000000000000000000000007E
S123B8C0FFFFFFFFFFFFFFFFFFFFFFFFFFFFFFFFFFFFFFFFFFFFFFFFFFFFFFFFFFFFFFFF84
S123B8E0FFFFFFFFFFFFFFFFFFFFFFFFFFFFFFFFFFFFFFFFFFFFFFFFFFFFFFFFFFFFFF0063
S123B900CC80381F8B108EB2BE8EB98710EE81EC81340610EFA18CB99725F11CAF7E886828
S123B92010CEB052CC80381F8BBD875EBDB96EBD896B7EB9008618B7E200B6ECE1B6ECE249
S123B9403D3D3DF6ECE2F7900E3D3D3DF6ECE2F7900D3D3D3DF6ECE2F7900C4FFB900D8946
S123B96000FB900E890047564756F7900A39CEB0508EE418C610BDF57133C84D30018CE463
S123B9801F23F1BDB93539AEB9900FAF31901FAFD190E2B051AC4F00000000000000000009
S123B9A0000000000000000000000000000000000000000000000000000000000000000083
S123B9C0FFFFFFFFFFFFFFFFFFFFFFFFFFFFFFFFFFFFFFFFFFFFFFFFFFFFFFFFFFFFFFFF83
S123B9E0FFFFFFFFFFFFFFFFFFFFFFFFFFFFFFFFFFFFFFFFFFFFFFFFFFFFFFFFFFFFFF0062
S123BA00000000000000000000000000000000000000000000000000000000000000000022
S123BA20000000000000000000000000000000000000000000000000000000000000000002
S123BA40FFFFFFFFFFFFFFFFFFFFFFFFFFFFFFFFFFFFFFFFFFFFFFFFFFFFFFFFFFFFFFFF02
S123BA60FFFFFFFFFFFFFFFFFFFFFFFFFFFFFFFFFFFFFFFFFFFFFFFFFFFFFFFFFFFFFFFFE2
S123BA800000000000000000000000000000000000000000000000000000000000000000A2
S123BAA0000000000000000000000000000000000000000000000000000000000000000082
S123BAC0FFFFFFFFFFFFFFFFFFFFFFFFFFFFFFFFFFFFFFFFFFFFFFFFFFFFFFFFFFFFFFFF82
S123BAE0FFFFFFFFFFFFFFFFFFFFFFFFFFFFFFFFFFFFFFFFFFFFFFFFFFFFFFFFFFFFFF0061
S123BB00000000000000000000000000000000000000000000000000000000000000000021
S123BB20000000000000000000000000000000000000000000000000000000000000000001
S123BB40FFFFFFFFFFFFFFFFFFFFFFFFFFFFFFFFFFFFFFFFFFFFFFFFFFFFFFFFFFFFFFFF01
S123BB60FFFFFFFFFFFFFFFFFFFFFFFFFFFFFFFFFFFFFFFFFFFFFFFFFFFFFFFFFFFFFFFFE1
S123BB800000000000000000000000000000000000000000000000000000000000000000A1
S123BBA0000000000000000000000000000000000000000000000000000000000000000081
S123BBC0FFFFFFFFFFFFFFFFFFFFFFFFFFFFFFFFFFFFFFFFFFFFFFFFFFFFFFFFFFFFFFFF81
S123BBE0FFFFFFFFFFFFFFFFFFFFFFFFFFFFFFFFFFFFFFFFFFFFFFFFFFFFFFFFFFFFFF0060
S123BC00000000000000000000000000000000000000000000000000000000000000000020
S123BC20000000000000000000000000000000000000000000000000000000000000000000
S123BC40FFFFFFFFFFFFFFFFFFFFFFFFFFFFFFFFFFFFFFFFFFFFFFFFFFFFFFFFFFFFFFFF00
S123BC60FFFFFFFFFFFFFFFFFFFFFFFFFFFFFFFFFFFFFFFFFFFFFFFFFFFFFFFFFFFFFFFFE0
S123BC800000000000000000000000000000000000000000000000000000000000000000A0
S123BCA0000000000000000000000000000000000000000000000000000000000000000080
S123BCC0FFFFFFFFFFFFFFFFFFFFFFFFFFFFFFFFFFFFFFFFFFFFFFFFFFFFFFFFFFFFFFFF80
S123BCE0FFFFFFFFFFFFFFFFFFFFFFFFFFFFFFFFFFFFFFFFFFFFFFFFFFFFFFFFFFFFFF005F
S123BD0000000000000000000000000000000000000000000000000000000000000000001F
S123BD200000000000000000000000000000000000000000000000000000000000000000FF
S123BD40FFFFFFFFFFFFFFFFFFFFFFFFFFFFFFFFFFFFFFFFFFFFFFFFFFFFFFFFFFFFFFFFFF
S123BD60FFFFFFFFFFFFFFFFFFFFFFFFFFFFFFFFFFFFFFFFFFFFFFFFFFFFFFFFFFFFFFFFDF
S123BD8000000000000000000000000000000000000000000000000000000000000000009F
S123BDA000000000000000000000000000000000000000000000000000000000000000007F
S123BDC0FFFFFFFFFFFFFFFFFFFFFFFFFFFFFFFFFFFFFFFFFFFFFFFFFFFFFFFFFFFFFFFF7F
S123BDE0FFFFFFFFFFFFFFFFFFFFFFFFFFFFFFFFFFFFFFFFFFFFFFFFFFFFFFFFFFFFFF005E
S123BE00E11E061E1E1E1E1EE1E1E1E1E1E1E1E11E1E1E1E1E1E1E1EE1E1E1E1E1E1E1E183
S123BE201E1E1A1E1E1E1E1EE1E1E1E1E1E1E1E11E1E1E1E1E1E1E1EE1E1E1E1E1E1E1E112
S123BE40E11E061E1E1E1E1EE1E1E1E1E1E1E1E11E1E1E1E1E1E1E1EE1E1E1E1E1E1E1E143
S123BE601E1E1E1E1E1E1E1EE1E1E1E1E1E1E1E11E1E1E1E1E1E1E1EE1E1E1E1E1E1E1E1CE
S123BE801E1E1E1E1E1E1E1EE1E1E1E1E1E1E1E11E1E1E1E1E1E1E1EE1E1E1E1E1E1E1E1AE
S123BEA01E1E1E1E1E1E1E1EE1E1E1E1E1E1E1E11E1E1E1E1E1E1E1EE1E1E1E1E1E1668169
S123BEC01E1E1E1E1E1E1E1EE1E1E1E1E1E1E1E11E1E1E1E1E1E1E1EE1E1E1E1E1E1E1E16E
S123BEE01E1E1E1E1E1E1E1EE1E1E1E1E1E1E1E11E1E1E1E1E1E1E1EE1E1E1E1E1E166C1E9
S123BF00E11E0E1E1E1E1E1EE1E1E1E1E1E1E1E11E1E1E1E1E1E1E1EE1E1E1E1E1E1E1E17A
S123BF201E1E1E1E1E1E1E1EE1E1E1E1E1E1E1E11E1E1E1E1E1E1E1EE1E1E1E1E1E1E1E10D
S123BF40E11E061E1E1E1E1EE1E1E1E1E1E1E1E11E1E1E1E1E1E1E1EE1E1E1E3E1E1E1E140
S123BF601E1E1E1E1E1E1E1EE1E1D01CD00800E80200973037976D46972020950C4394FBCB
S123BF80000B050B05021E1EE1E1E1E100802E0000800000001E1E1EE1E1E1E1E1E1E1E12B
S123BFA01E1E1E1E1E1E1E1EE1E1E1E1E1E1E1E11E1E1E1E1E1E1E1EE1E1E1E1E1E166A940
S123BFC01E1E1E1E1E1E1E1EE1E1E1E1E1E1E1E11E1E1E1E1E1E1E1EE1E1E1E1E1E1E1E16D
S123BFE01E1E1E1E1E1E1E1EE1E1E1E1E1E1E1E11E1E1E1E1E1E1E1EE1E1E1E1E1E166C1E8
S123F000B6800397028688B780009700139603A78020F9B6800397028688B7800097001391
S123F020960320FBB68003970286A8B78000970013A680970320F9B68003970286A8B78027
S123F04000970013A684970320F986E8B780009700139603A78020F986F8B780009700139E
S123F060A680970320F9860CB78000970020FEB680029703861CB78000970020FE8658B740
S123F0808000970020FE8678B78000970020FE86D0B780009700D600C50126FAF7800610E0
S123F0A08E00011700013912121212313F26F839326CD600F78006B6800081882707B680C9
S123F0C00081E8260AF68006C45CF780062020B6800081A82707B6800081F8260AF6800652
S123F0E0C45CF780062008F68006C418F78006391A50861FB7E2028610B7E2008EE4006F7F
S123F100808CE40826F9B7E41810CEBF80BDF1E5BDF15DBDF4C68640B4E20081002712BD1C
S123F120F20DB6800681002706BDF413BDF306200EBDF4D68607B78006B78007BDF306B63F
S123F1408006810026CA9601B7800286A6B7E20E8695B7E1008630B7E2007E800E86E81F76
S123F1608BBDF08F867FB7E20E86CCB7E20B860EB7E20C861FB7E2038630B7E2007FE206F2
S123F1807FE2077FE2047FE205CC1388F7E208B7E20986FFB7ECE18EEC006F808CECE0265E
S123F1A0F9BDF1BB8603B7E1007F80067F80077F80027F80038601B7BF8C398EEC80861068
S123F1C0A7808CECA026F78EECA08663A7808CECC026F7C620B6ECE0108E000CBDF0A75A90
S123F1E0C10026F1397FBF85B6BF85BAE200B7E2008E0000867FA7808C800026F97CBF8563
S123F200B6BF85810426E18610B7E20039BDF066B68006810027031600917FBF858E80008A
S123F220BF8004B6BF854848B7BF80108EFB80BDF38CB680068100270316006FB6BF81B799
S123F2408002B6BF82B78003B6BF8C2703BDF425BDF3ACB6800681002702204FB6BF8C271D
S123F2600A3410BDF4377FBF8C3510BF80047C8003B68003810626D07C8002B68002B1BFA7
S123F28083220CBDF3F1B6800681002702201CB68002B1BF8323AB7CBF85B6BF8581022799
S123F2A0078CBE001026FF7BBDF2AFBDF4D639108EFB887FBF80BDF38CB680068100270329
S123F2C01600428E0000BF8004B6BF81B78002B6BF82B78003BDF3ACB6800681002702203F
S123F2E024108E802E10BFBF8D108E00008E8011A6A0A780BCBF8D26F78E0000867FA78076
S123F3008C020026F939B6800781012608CC7A9EFDBF8A201681062608CC387AFDBF8A201D
S123F3200A81072606CC2A7AFDBF8A867FB7BF85BDF33C7ABF85B6BF8526F539FCBF8AB761
S123F340BF88F7BF895FF7BF871F988A18C680F5BF86260578BF88200778BF88240284F73D
S123F360C680F5BF86260578BF89200778BF89240284EFB7E201108E0100313F26FC7CBF98
S123F38086F6BF875CC1071023FFBB39B6BF8030A6A680B7BF81B78002A680B7BF82A680F8
S123F3A0B7BF83A684B7BF84BDF3F139860AB78001BE8004BDF000B6800681002708B6BF3A
S123F3C08C2703BDF4377A8001B680012707B68006810026DCB6800681002714BDF086BD84
S123F3E0F07DB6BF8C2703BDF437BE8004BDF000398602B78001BDF06FB68006810027069B
S123F400BDF0667A8001B680012707B68006810026E4398601B780078610F58006270586ED
S123F42006B78007398EBF8D108E8000A6A0A780108C800826F6398E8000108EBF8DA6A02F
S123F440A7808C800826F739860AB78001BE8004BDF0007A8001B680012707B68006810043
S123F46026EBB680068100270CBDF086BDF07DBE8004BDF00039860AB78001BE8004BDF04B
S123F480247A8001B680012707B68006810026EBB680068100270CBDF086BDF07DBE800487
S123F4A0BDF024398602B78001BDF06FB6800681002706BDF0667A8001B680012707B680CF
S123F4C006810026E439B6E20084EFB7E200108EFFFFBDF0A739B6E2008A10B7E20039CCC1
S123F4E01388B7E2091CBF032E27040A2F20040A300C360A33963727034A9737963127037E
S123F5004A9731963227034A9732DC342705830001DD343B408B0934028EF94D3A3AEC8402
S123F5206DE42B0644566AE42AFA326139CC1388F7E208B7E20986A6B7E20ECC80381F8B82
S123F54039867FB7E20E8603B7E1007FE20012128630B7E2008618B7E20F39A680A7C03190
S123F5603F26F839A684E6C4A7C0E780313F26F439C11027037EFC91F7E200C6B0BDF5DCA9
S123F5808D3C108E00008D368D348D328D30108C00002718108C0FA02412108C008525035B
S123F5A05C20DA108C008022035A20D1C07AE7C8185FBDF5DCE71039121212121212B6EC39
S123F5C0E28D1931212714B6ECE2819025F38D0C31212707B6ECE2817022F33986FFA784D9
S123F5E0A710E784E71839A7C4A758E7C0E7C8EF391A5035403506E78883A788A3E78884F4
S123F600A788A43506E78881A788A1E78882A788A21CAF6EC4FFFFFFFFFFFFFFFFFFFFFF64
S123F620FFFFFFFFFFFFFFFFFFFFFFFFFFFFFFFFFFFFFFFFFFFFFFFFFFFFFFFFFFFFFFFFE6
S123F640FFFFFFFFFFFFFFFFFFFFFFFFFFFFFFFFFFFFFFFFFFFFFFFFFFFFFFFFFFFFFFFFC6
S123F660FFFFFFFFFFFFFFFFFFFFFFFFFFFFFFFFFFFFFFFFFFFFFFFFFFFFFFFFFFFFFFFFA6
S123F680FFFFFFFFFFFFFFFFFFFFFFFFFFFFFFFFFFFFFFFFFFFFFFFFFFFFFFFFFFFFFFFF86
S123F6A0FFFFFFFFFFFFFFFFFFFFFFFFFFFFFFFFFFFFFFFFFFFFFFFFFFFFFFFFFFFFFFFF66
S123F6C0FFFFFFFFFFFFFFFFFFFFFFFFFFFFFFFFFFFFFFFFFFFFFFFFFFFFFFFFFF1A50ECED
S123F6E062A7A8C2A7A8C1E7A8C3E7A8C41CAF3506EDE439FFFFFFFFFFFFFFFFFFFFFFFFDA
S123F700FFFFFFFFFFFFFFFFFFFFFFFFFFFFFFFFFFFFFFFFFFFFFFFFFFFFFFFFFFFFFFFF05
S123F720FFFFFFFFFFFFFFFFFFFFFFFFFFFFFFFFFFFFFFFFFFFFFFFFFFFFFFFFFFFFFFFFE5
S123F740FFFFFFFFFFFFFFFFFFFFFFFFFFFFFFFFFFFFFFFFFFFFFFFFFFFFFFFFFFFFFFFFC5
S123F760FFFFFFFFFFFFFFFFFFFFFFFFFFFFFFFFFFFFFFFFFFFFFFFFFFFFFFFFFF000000A2
S123F780000000000001010101010101020202020203030303040405050606070708080903
S123F7A0090A0A0B0B0C0C0D0D0E0E0F0F101112131415161718191A1B1C1D1E1F202122CB
S123F7C0232425262728292A2B2C2D2E2F303132333435363738393A3B3C3D3E3F404243D3
S123F7E04546484A4C4E50525456585A5C5E616366696C6F7275787B7F7F7F7F7FFFFF8055
S123F8000040002EE02000177010000BB808000666051E04100333028F02190199014701AC
S123F8200600CF00A30083006800530042003600290021001A00140010000D000A000800EF
S123F8400600050004000300020001000000020406080A0C0E10121416181A1C1E20222439
S123F86026282A2C2E30323436383A3C3E40424446484A4C4E50525456585A5C5E606264E4
S123F88066686A6C6E70727475767778797A79787776757472706E6C6A68666462605E5C94
S123F8A05A58565452504E4C4A48464442403E3C3A38363432302E2C2A28262422201E1CE4
S123F8C01A18161412100E0C0A0806040200FEFCFAF8F6F4F2F0EEECEAE8E6E4E2E0DEDCC4
S123F8E0DAD8D6D4D2D0CECCCAC8C6C4C2C0BEBCBAB8B6B4B2B0AEACAAA8A6A4A2A09E9CA4
S123F9009A98969492908E8C8B8A898887868788898A8B8C8E90929496989A9C9EA0A2A4B3
S123F920A6A8AAACAEB0B2B4B6B8BABCBEC0C2C4C6C8CACCCED0D2D4D6D8DADCDEE0E2E423
S123F940E6E8EAECEEF0F2F4F6F8FAFCFE49114944497649A949DC4A104A434A774AAA4AB6
S123F960DE4B124B464B7B4BAF4BE34C184C4D4C824CB74CEC4D224D574D8D4DC34DF94E32
S123F9802F4E654E9B4ED24F094F404F774FAE4FE5501D5054508C50C450FC5134516C51BA
S123F9A0A551DE5216524F528952C252FB5335536F53A953E3541D5457549254CC550755DB
S123F9C042557E55B955F45630566C56A856E45720575D579957D658135850588E58CB597A
S123F9E0095947598459C35A015A3F5A7E5ABD5AFC5B3B5B7A5BBA5BF95C395C795CBA5C78
S123FA00FA5D3A5D7B5DBC5DFD5E3E5E805EC15F035F455F875FC9600C604F609160D461B8
S123FA2018615B619F61E26226626B62AF62F36338637D63C26407644D649264D8651E651A
S123FA406465AB65F16638667F66C6670D6755679D67E4682D687568BD6906694F69986982
S123FA60E16A2B6A756ABE6B096B536B9D6BE86C336C7E6CC96D156D616DAD6DF96E456EC9
S123FA80916EDE6F2B6F786FC67013706170AF70FD714C719A71E97238728872D7732773D3
S123FAA07773C77417746874B9750A755B75AC75FE765076A276F47747779A77ED7840786F
S123FAC09378E7793B798F79E47A387A8D7AE27B377B8D7BE37C397C8F7CE57D3C7D937D83
S123FAE0EA7E417E997EF17F497FA17FFA805380AC8105815F81B98213826D82C7832283DE
S123FB007D83D98434849084EC854885A58601865E86BC8719877787D58833889288F18957
S123FB205089AF8A0E8A6E8ACE8B2F8B8F8BF08C518CB38D148D768DD88E3B8E9E8F018FC9
S123FB40648FC7902B908F90F4915891BDFC60DAF266B6BEE0FEE6EE3E9C7A9E8E1C2A3A9E
S123FB60CE0A7C1002801A3810030111060412090715050E16080C17000F14020D130A0B35
S123FB800000010502050A050B050B052005220502000E041C002804360042040F001B04D3
S123FBA02900350443004F04140517052305260537053A0518051B051C051F0527052A0569
S123FBC02B052E053B053E050C051F052305360537054A0500000002082004001000400694
S123FBE018600102040810204080010204E69D7BFEFDFBFEFEFDFDFB010101020202020390
S123FC00030303030404040404040505050505050506060606060606060707070707070738
S123FC200707080808080808080809090909090909090A0A0A0A0A0A0A0B0B0B0B0B0B0C96
S123FC400C0C0C0C0D0D0D0D0D0E0E0E0E0F0F0F0F0F1010101011111112121313141415B2
S123FC601617191B1E212326292C2F32363B4148515A646E797F7F7F7F7F7F7F7F7F7F4FAC
S123FC808EC000A1801026F4674C811026F57EC0108602B78003867FB78001CCFDB7FDBFDF
S123FCA08ABDF33C7A8001B6800126F57A8003B6800326E27EF0F0FFFFFFFFFFFFFFFFFFEA
S123FCC0FFFFFFFFFFFFFFFFFFFFFFFFFFFFFFFFFFFFFFFFFFFFFFFFFFFFFFFFFFFFFFFF40
S123FCE0FFFFFFFFFFFFFFFFFFFFFFFFFFFFFFFFFFFFFFFFFFFFFFFFFFFFFFFFFFFFFFFF20
S123FD00FFFFFFFFFFFFFFFFFFFFFFFFFFFFFFFFFFFFFFFFFFFFFFFFFFFFFFFFFFFFFFFFFF
S123FD20FFFFFFFFFFFFFFFFFFFFFFFFFFFFFFFFFFFFFFFFFFFFFFFFFFFFFFFFFFFFFFFFDF
S123FD40FFFFFFFFFFFFFFFFFFFFFFFFFFFFFFFFFFFFFFFFFFFFFFFFFFFFFFFFFFFFFFFFBF
S123FD60FFFFFFFFFFFFFFFFFFFFFFFFFFFFFFFFFFFFFFFFFFFFFFFFFFFFFFFFFFFFFFFF9F
S123FD80FFFFFFFFFFFFFFFFFFFFFFFFFFFFFFFFFFFFFFFFFFFFFFFFFFFFFFFFFFFFFFFF7F
S123FDA0FFFFFFFFFFFFFFFFFFFFFFFFFFFFFFFFFFFFFFFFFFFFFFFFFFFFFFFFFFFFFFFF5F
S123FDC0FFFFFFFFFFFFFFFFFFFFFFFFFFFFFFFFFFFFFFFFFFFFFFFFFFFFFFFFFFFFFFFF3F
S123FDE0FFFFFFFFFFFFFFFFFFFFFFFFFFFFFFFFFFFFFFFFFFFFFFFFFFFFFFFFFFFFFFFF1F
S123FE00FFFFFFFFFFFFFFFFFFFFFFFFFFFFFFFFFFFFFFFFFFFFFFFFFFFFFFFFFFFFFFFFFE
S123FE20FFFFFFFFFFFFFFFFFFFFFFFFFFFFFFFFFFFFFFFFFFFFFFFFFFFFFFFFFFFFFFFFDE
S123FE40FFFFFFFFFFFFFFFFFFFFFFFFFFFFFFFFFFFFFFFFFFFFFFFFFFFFFFFFFFFFFFFFBE
S123FE60FFFFFFFFFFFFFFFFFFFFFFFFFFFFFFFFFFFFFFFFFFFFFFFFFFFFFFFFFFFFFFFF9E
S123FE80FFFFFFFFFFFFFFFFFFFFFFFFFFFFFFFFFFFFFFFFFFFFFFFFFFFFFFFFFFFFFFFF7E
S123FEA0FFFFFFFFFFFFFFFFFFFFFFFFFFFFFFFFFFFFFFFFFFFFFFFFFFFFFFFFFFFFFFFF5E
S123FEC0FFFFFFFFFFFFFFFFFFFFFFFFFFFFFFFFFFFFFFFFFFFFFFFFFFFFFFFFFFFFFFFF3E
S123FEE0FFFFFFFFFFFFFFFFFFFFFFFFFFFFFFFFFFFFFFFFFFFFFFFFFFFFFFFFFFFFFFFF1E
S123FF00FFFFFFFFFFFFFFFFFFFFFFFFFFFFFFFFFFFFFFFFFFFFFFFFFFFFFFFFFFFFFFFFFD
S123FF20FFFFFFFFFFFFFFFFFFFFFFFFFFFFFFFFFFFFFFFFFFFFFFFFFFFFFFFFFFFFFFFFDD
S123FF40FFFFFFFFFFFFFFFFFFFFFFFFFFFFFFFFFFFFFFFFFFFFFFFFFFFFFFFFFFFFFFFFBD
S123FF60FFFFFFFFFFFFFFFFFFFFFFFFFFFFFFFFFFFFFFFFFFFFFFFFFFFFFFFFFFFFFFFF9D
S123FF80FFFFFFFFFFFFFFFFFFFFFFFFFFFFFFFFFFFFFFFFFFFFFFFFFFFFFFFFFFFFFFFF7D
S123FFA0FFFFFFFFFFFFFFFFFFFFFFFFFFFFFFFFFFFFFFFFFFFFFFFFFFFFFFFFFFFFFFFF5D
S123FFC0FFFFFFFFFFFFFFFFFFFFFFFFFFFFFFFFFFFFFFFFFFFFFFFFFFFFFFFFFFFFFFFF3D
S123FFE0FFFFFFFFFFFFFFFFFFFFFFFFFFFFFFFFFC7FFC7FFC7F800B8008FC7FF0B0FC7FF3
